 dt_socket

 Timestamp is 6710e055 (Thu Oct 17 10:00:53 2024)

 Preferred load address is 10000000

 Start         Length     Name                   Class
 0001:00000000 000021e9H .text$mn                CODE
 0002:00000000 00000118H .idata$5                DATA
 0002:00000118 00000008H .00cfg                  DATA
 0002:00000120 00000004H .CRT$XCA                DATA
 0002:00000124 00000004H .CRT$XCZ                DATA
 0002:00000128 00000004H .CRT$XIA                DATA
 0002:0000012c 00000004H .CRT$XIZ                DATA
 0002:00000130 00000004H .CRT$XPA                DATA
 0002:00000134 00000004H .CRT$XPZ                DATA
 0002:00000138 00000004H .CRT$XTA                DATA
 0002:0000013c 00000004H .CRT$XTZ                DATA
 0002:00000140 00000000H .gfids$y                DATA
 0002:00000140 00000b40H .rdata                  DATA
 0002:00000c80 00000000H .rdata$CastGuardVftablesA DATA
 0002:00000c80 00000000H .rdata$CastGuardVftablesC DATA
 0002:00000c80 00000004H .rdata$sxdata           DATA
 0002:00000c84 0000006cH .rdata$voltmd           DATA
 0002:00000cf0 000002f0H .rdata$zzzdbg           DATA
 0002:00000fe0 00000004H .rtc$IAA                DATA
 0002:00000fe4 00000004H .rtc$IZZ                DATA
 0002:00000fe8 00000004H .rtc$TAA                DATA
 0002:00000fec 00000004H .rtc$TZZ                DATA
 0002:00000ff0 00000090H .xdata$x                DATA
 0002:00001080 00000058H .edata                  DATA
 0002:000010d8 0000008cH .idata$2                DATA
 0002:00001164 00000014H .idata$3                DATA
 0002:00001178 00000118H .idata$4                DATA
 0002:00001290 000003aaH .idata$6                DATA
 0003:00000000 00000028H .data                   DATA
 0003:00000028 000003b4H .bss                    DATA
 0004:00000000 00000060H .rsrc$01                DATA
 0004:00000060 00000320H .rsrc$02                DATA

  Address         Publics by Value              Rva+Base       Lib:Object

 0000:00000000       ___AbsoluteZero            00000000     <absolute>
 0000:00000000       ___arm64x_extra_rfe_table  00000000     <absolute>
 0000:00000000       ___arm64x_extra_rfe_table_size 00000000     <absolute>
 0000:00000000       ___arm64x_native_entrypoint 00000000     <absolute>
 0000:00000000       ___arm64x_redirection_metadata 00000000     <absolute>
 0000:00000000       ___arm64x_redirection_metadata_count 00000000     <absolute>
 0000:00000000       ___dynamic_value_reloc_table 00000000     <absolute>
 0000:00000000       ___enclave_config          00000000     <absolute>
 0000:00000000       ___guard_check_icall_a64n_fptr 00000000     <absolute>
 0000:00000000       ___guard_eh_cont_count     00000000     <absolute>
 0000:00000000       ___guard_eh_cont_table     00000000     <absolute>
 0000:00000000       ___guard_fids_count        00000000     <absolute>
 0000:00000000       ___guard_fids_table        00000000     <absolute>
 0000:00000000       ___guard_iat_count         00000000     <absolute>
 0000:00000000       ___guard_iat_table         00000000     <absolute>
 0000:00000000       ___guard_longjmp_count     00000000     <absolute>
 0000:00000000       ___guard_longjmp_table     00000000     <absolute>
 0000:00000000       ___hybrid_auxiliary_delayload_iat 00000000     <absolute>
 0000:00000000       ___hybrid_auxiliary_delayload_iat_copy 00000000     <absolute>
 0000:00000000       ___hybrid_auxiliary_iat    00000000     <absolute>
 0000:00000000       ___hybrid_auxiliary_iat_copy 00000000     <absolute>
 0000:00000000       ___hybrid_code_map         00000000     <absolute>
 0000:00000000       ___hybrid_code_map_count   00000000     <absolute>
 0000:00000000       ___hybrid_image_info_bitfield 00000000     <absolute>
 0000:00000000       ___x64_code_ranges_to_entry_points 00000000     <absolute>
 0000:00000000       ___x64_code_ranges_to_entry_points_count 00000000     <absolute>
 0000:00000001       ___safe_se_handler_count   00000001     <absolute>
 0000:00000100       ___guard_flags             00000100     <absolute>
 0000:00000000       ___ImageBase               10000000     <linker-defined>
 0001:00000000       ___local_stdio_printf_options 10001000 f i socketTransport.obj
 0001:00000006       __vfprintf_l               10001006 f i socketTransport.obj
 0001:0000002a       __vsnprintf_l              1000102a f i socketTransport.obj
 0001:0000005d       _fprintf                   1000105d f i socketTransport.obj
 0001:000001e7       _jdwpTransport_OnLoad@16   100011e7 f   socketTransport.obj
 0001:00000e17       _sprintf                   10001e17 f i socketTransport.obj
 0001:00000e31       _DllMain@12                10001e31 f   socket_md.obj
 0001:00000e82       _dbgsysAccept              10001e82 f   socket_md.obj
 0001:00000e95       _dbgsysBind                10001e95 f   socket_md.obj
 0001:00000ea8       _dbgsysConfigureBlocking   10001ea8 f   socket_md.obj
 0001:00000ed5       _dbgsysConnect             10001ed5 f   socket_md.obj
 0001:00000f1a       _dbgsysCurrentTimeMillis   10001f1a f   socket_md.obj
 0001:00000fb3       _dbgsysFinishConnect       10001fb3 f   socket_md.obj
 0001:0000104f       _dbgsysGetHostByName       1000204f f   socket_md.obj
 0001:0000105a       _dbgsysGetLastIOError      1000205a f   socket_md.obj
 0001:0000109a       _dbgsysGetSocketName       1000209a f   socket_md.obj
 0001:000010ad       _dbgsysHostToNetworkLong   100020ad f   socket_md.obj
 0001:000010b8       _dbgsysHostToNetworkShort  100020b8 f   socket_md.obj
 0001:000010c3       _dbgsysInetAddr            100020c3 f   socket_md.obj
 0001:000010ce       _dbgsysListen              100020ce f   socket_md.obj
 0001:000010dd       _dbgsysNetworkToHostLong   100020dd f   socket_md.obj
 0001:000010e8       _dbgsysNetworkToHostShort  100020e8 f   socket_md.obj
 0001:000010f3       _dbgsysPoll                100020f3 f   socket_md.obj
 0001:000011b8       _dbgsysRecv                100021b8 f   socket_md.obj
 0001:000011cf       _dbgsysSend                100021cf f   socket_md.obj
 0001:000011e6       _dbgsysSetSocketOption     100021e6 f   socket_md.obj
 0001:000012ce       _dbgsysSocket              100022ce f   socket_md.obj
 0001:000012f7       _dbgsysSocketClose         100022f7 f   socket_md.obj
 0001:0000133d       _dbgsysTlsAlloc            1000233d f   socket_md.obj
 0001:00001343       _dbgsysTlsGet              10002343 f   socket_md.obj
 0001:0000134e       _dbgsysTlsPut              1000234e f   socket_md.obj
 0001:0000135d       ___WSAFDIsSet@8            1000235d f   ws2_32:WS2_32.dll
 0001:00001363       ___raise_securityfailure   10002363 f   MSVCRT:gs_report.obj
 0001:0000138b       ___report_gsfailure        1000238b f   MSVCRT:gs_report.obj
 0001:00001485       ___report_rangecheckfailure 10002485 f   MSVCRT:gs_report.obj
 0001:00001491       ___report_securityfailure  10002491 f   MSVCRT:gs_report.obj
 0001:00001560       @__security_check_cookie@4 10002560 f   MSVCRT:secchk.obj
 0001:00001570       __alldiv                   10002570 f   MSVCRT:lldiv.obj
 0001:0000195a       __DllMainCRTStartup@12     1000295a f   MSVCRT:dll_dllmain.obj
 0001:000019ca       ___security_init_cookie    100029ca f   MSVCRT:gs_support.obj
 0001:00001a15       ?__scrt_initialize_type_info@@YAXXZ 10002a15 f   MSVCRT:tncleanup.obj
 0001:00001a21       ?__scrt_uninitialize_type_info@@YAXXZ 10002a21 f   MSVCRT:tncleanup.obj
 0001:00001a2d       ___local_stdio_scanf_options 10002a2d f i MSVCRT:default_local_stdio_options.obj
 0001:00001a33       ___scrt_initialize_default_local_stdio_options 10002a33 f   MSVCRT:default_local_stdio_options.obj
 0001:00001a94       ___scrt_acquire_startup_lock 10002a94 f   MSVCRT:utility.obj
 0001:00001ac6       ___scrt_dllmain_after_initialize_c 10002ac6 f   MSVCRT:utility.obj
 0001:00001af1       ___scrt_dllmain_before_initialize_c 10002af1 f   MSVCRT:utility.obj
 0001:00001aff       ___scrt_dllmain_crt_thread_attach 10002aff f   MSVCRT:utility.obj
 0001:00001b1e       ___scrt_dllmain_crt_thread_detach 10002b1e f   MSVCRT:utility.obj
 0001:00001b2b       ___scrt_dllmain_exception_filter 10002b2b f   MSVCRT:utility.obj
 0001:00001b5f       ___scrt_dllmain_uninitialize_c 10002b5f f   MSVCRT:utility.obj
 0001:00001b82       ___scrt_dllmain_uninitialize_critical 10002b82 f   MSVCRT:utility.obj
 0001:00001b8f       ___scrt_initialize_crt     10002b8f f   MSVCRT:utility.obj
 0001:00001bc8       ___scrt_initialize_onexit_tables 10002bc8 f   MSVCRT:utility.obj
 0001:00001c4f       ___scrt_is_nonwritable_in_current_image 10002c4f f   MSVCRT:utility.obj
 0001:00001ce3       ___scrt_release_startup_lock 10002ce3 f   MSVCRT:utility.obj
 0001:00001d00       ___scrt_uninitialize_crt   10002d00 f   MSVCRT:utility.obj
 0001:00001d28       ___scrt_get_dyn_tls_init_callback 10002d28 f   MSVCRT:dyn_tls_init.obj
 0001:00001d2e       ___scrt_fastfail           10002d2e f   MSVCRT:utility_desktop.obj
 0001:00001e49       __crt_debugger_hook        10002e49 f   MSVCRT:utility_desktop.obj
 0001:00001e51       __RTC_Initialize           10002e51 f   MSVCRT:initsect.obj
 0001:00001e7d       __RTC_Terminate            10002e7d f   MSVCRT:initsect.obj
 0001:00001eb0       __SEH_prolog4              10002eb0 f   MSVCRT:sehprolg4.obj
 0001:00001ef5       __except_handler4          10002ef5 f   MSVCRT:chandler4gs.obj
 0001:00001f24       @_guard_check_icall_nop@4  10002f24 f i MSVCRT:guard_support.obj
 0001:00001f27       ___isa_available_init      10002f27 f   MSVCRT:cpu_disp.obj
 0001:000020fb       __get_startup_argv_mode    100030fb f   MSVCRT:argv_mode.obj
 0001:000020ff       ___scrt_is_ucrt_dll_in_use 100030ff f   MSVCRT:ucrt_detection.obj
 0001:0000210b       _memcpy                    1000310b f   vcruntime:VCRUNTIME140.dll
 0001:00002111       _memset                    10003111 f   vcruntime:VCRUNTIME140.dll
 0001:00002117       _strchr                    10003117 f   vcruntime:VCRUNTIME140.dll
 0001:0000211d       ___std_type_info_destroy_list 1000311d f   vcruntime:VCRUNTIME140.dll
 0001:00002123       __except_handler4_common   10003123 f   vcruntime:VCRUNTIME140.dll
 0001:00002129       _strcat                    10003129 f   ucrt:api-ms-win-crt-string-l1-1-0.dll
 0001:0000212f       _strcpy                    1000312f f   ucrt:api-ms-win-crt-string-l1-1-0.dll
 0001:00002135       _strlen                    10003135 f   ucrt:api-ms-win-crt-string-l1-1-0.dll
 0001:0000213b       __initterm                 1000313b f   ucrt:api-ms-win-crt-runtime-l1-1-0.dll
 0001:00002141       __initterm_e               10003141 f   ucrt:api-ms-win-crt-runtime-l1-1-0.dll
 0001:00002147       __seh_filter_dll           10003147 f   ucrt:api-ms-win-crt-runtime-l1-1-0.dll
 0001:0000214d       __configure_narrow_argv    1000314d f   ucrt:api-ms-win-crt-runtime-l1-1-0.dll
 0001:00002153       __initialize_narrow_environment 10003153 f   ucrt:api-ms-win-crt-runtime-l1-1-0.dll
 0001:00002159       __initialize_onexit_table  10003159 f   ucrt:api-ms-win-crt-runtime-l1-1-0.dll
 0001:0000215f       __execute_onexit_table     1000315f f   ucrt:api-ms-win-crt-runtime-l1-1-0.dll
 0001:00002165       __cexit                    10003165 f   ucrt:api-ms-win-crt-runtime-l1-1-0.dll
 0001:0000216b       ___acrt_initialize         1000316b f   MSVCRT:ucrt_stubs.obj
 0001:0000216b       ___acrt_thread_attach      1000316b f   MSVCRT:ucrt_stubs.obj
 0001:0000216b       ___acrt_thread_detach      1000316b f   MSVCRT:ucrt_stubs.obj
 0001:0000216b       ___acrt_uninitialize       1000316b f   MSVCRT:ucrt_stubs.obj
 0001:0000216b       ___acrt_uninitialize_critical 1000316b f   MSVCRT:ucrt_stubs.obj
 0001:0000216b       ___scrt_stub_for_acrt_initialize 1000316b f   MSVCRT:ucrt_stubs.obj
 0001:0000216b       ___scrt_stub_for_acrt_thread_attach 1000316b f   MSVCRT:ucrt_stubs.obj
 0001:0000216b       ___scrt_stub_for_acrt_thread_detach 1000316b f   MSVCRT:ucrt_stubs.obj
 0001:0000216b       ___scrt_stub_for_acrt_uninitialize 1000316b f   MSVCRT:ucrt_stubs.obj
 0001:0000216b       ___scrt_stub_for_acrt_uninitialize_critical 1000316b f   MSVCRT:ucrt_stubs.obj
 0001:0000216b       ___vcrt_initialize         1000316b f   MSVCRT:ucrt_stubs.obj
 0001:0000216b       ___vcrt_thread_attach      1000316b f   MSVCRT:ucrt_stubs.obj
 0001:0000216b       ___vcrt_thread_detach      1000316b f   MSVCRT:ucrt_stubs.obj
 0001:0000216b       ___vcrt_uninitialize       1000316b f   MSVCRT:ucrt_stubs.obj
 0001:0000216b       ___vcrt_uninitialize_critical 1000316b f   MSVCRT:ucrt_stubs.obj
 0001:0000216e       ___scrt_stub_for_is_c_termination_complete 1000316e f   MSVCRT:ucrt_stubs.obj
 0001:0000216e       __is_c_termination_complete 1000316e f   MSVCRT:ucrt_stubs.obj
 0001:00002171       __filter_x86_sse2_floating_point_exception 10003171 f   MSVCRT:x86_exception_filter.obj
 0001:00002171       __filter_x86_sse2_floating_point_exception_default 10003171 f   MSVCRT:x86_exception_filter.obj
 0002:00000000       __imp__QueryPerformanceCounter@4 10004000     kernel32:KERNEL32.dll
 0002:00000004       __imp__IsDebuggerPresent@0 10004004     kernel32:KERNEL32.dll
 0002:00000008       __imp__InitializeSListHead@4 10004008     kernel32:KERNEL32.dll
 0002:0000000c       __imp__GetSystemTimeAsFileTime@4 1000400c     kernel32:KERNEL32.dll
 0002:00000010       __imp__GetCurrentThreadId@0 10004010     kernel32:KERNEL32.dll
 0002:00000014       __imp__GetCurrentProcessId@0 10004014     kernel32:KERNEL32.dll
 0002:00000018       __imp__IsProcessorFeaturePresent@4 10004018     kernel32:KERNEL32.dll
 0002:0000001c       __imp__TerminateProcess@8  1000401c     kernel32:KERNEL32.dll
 0002:00000020       __imp__GetCurrentProcess@0 10004020     kernel32:KERNEL32.dll
 0002:00000024       __imp__SetUnhandledExceptionFilter@4 10004024     kernel32:KERNEL32.dll
 0002:00000028       __imp__UnhandledExceptionFilter@4 10004028     kernel32:KERNEL32.dll
 0002:0000002c       __imp__SystemTimeToFileTime@8 1000402c     kernel32:KERNEL32.dll
 0002:00000030       __imp__GetSystemTime@4     10004030     kernel32:KERNEL32.dll
 0002:00000034       __imp__TlsSetValue@8       10004034     kernel32:KERNEL32.dll
 0002:00000038       __imp__TlsGetValue@4       10004038     kernel32:KERNEL32.dll
 0002:0000003c       __imp__TlsAlloc@0          1000403c     kernel32:KERNEL32.dll
 0002:00000040       __imp__SetHandleInformation@12 10004040     kernel32:KERNEL32.dll
 0002:00000044       \177KERNEL32_NULL_THUNK_DATA 10004044     kernel32:KERNEL32.dll
 0002:00000048       __imp____std_type_info_destroy_list 10004048     vcruntime:VCRUNTIME140.dll
 0002:0000004c       __imp__strchr              1000404c     vcruntime:VCRUNTIME140.dll
 0002:00000050       __imp__memset              10004050     vcruntime:VCRUNTIME140.dll
 0002:00000054       __imp__memcpy              10004054     vcruntime:VCRUNTIME140.dll
 0002:00000058       __imp___except_handler4_common 10004058     vcruntime:VCRUNTIME140.dll
 0002:0000005c       \177VCRUNTIME140_NULL_THUNK_DATA 1000405c     vcruntime:VCRUNTIME140.dll
 0002:00000060       __imp__send@16             10004060     ws2_32:WS2_32.dll
 0002:00000064       __imp__select@20           10004064     ws2_32:WS2_32.dll
 0002:00000068       __imp__recv@16             10004068     ws2_32:WS2_32.dll
 0002:0000006c       __imp__ntohs@4             1000406c     ws2_32:WS2_32.dll
 0002:00000070       __imp__ntohl@4             10004070     ws2_32:WS2_32.dll
 0002:00000074       __imp__listen@8            10004074     ws2_32:WS2_32.dll
 0002:00000078       __imp__setsockopt@20       10004078     ws2_32:WS2_32.dll
 0002:0000007c       __imp__htons@4             1000407c     ws2_32:WS2_32.dll
 0002:00000080       __imp__htonl@4             10004080     ws2_32:WS2_32.dll
 0002:00000084       __imp____WSAFDIsSet@8      10004084     ws2_32:WS2_32.dll
 0002:00000088       __imp__getsockopt@20       10004088     ws2_32:WS2_32.dll
 0002:0000008c       __imp__getsockname@12      1000408c     ws2_32:WS2_32.dll
 0002:00000090       __imp__ioctlsocket@12      10004090     ws2_32:WS2_32.dll
 0002:00000094       __imp__connect@12          10004094     ws2_32:WS2_32.dll
 0002:00000098       __imp__closesocket@4       10004098     ws2_32:WS2_32.dll
 0002:0000009c       __imp__bind@12             1000409c     ws2_32:WS2_32.dll
 0002:000000a0       __imp__accept@12           100040a0     ws2_32:WS2_32.dll
 0002:000000a4       __imp__WSASendDisconnect@8 100040a4     ws2_32:WS2_32.dll
 0002:000000a8       __imp__WSAGetLastError@0   100040a8     ws2_32:WS2_32.dll
 0002:000000ac       __imp__WSACleanup@0        100040ac     ws2_32:WS2_32.dll
 0002:000000b0       __imp__WSAStartup@8        100040b0     ws2_32:WS2_32.dll
 0002:000000b4       __imp__getprotobyname@4    100040b4     ws2_32:WS2_32.dll
 0002:000000b8       __imp__gethostbyname@4     100040b8     ws2_32:WS2_32.dll
 0002:000000bc       __imp__inet_addr@4         100040bc     ws2_32:WS2_32.dll
 0002:000000c0       __imp__socket@12           100040c0     ws2_32:WS2_32.dll
 0002:000000c4       \177WS2_32_NULL_THUNK_DATA 100040c4     ws2_32:WS2_32.dll
 0002:000000c8       __imp__atoi                100040c8     ucrt:api-ms-win-crt-convert-l1-1-0.dll
 0002:000000cc       \177api-ms-win-crt-convert-l1-1-0_NULL_THUNK_DATA 100040cc     ucrt:api-ms-win-crt-convert-l1-1-0.dll
 0002:000000d0       __imp___cexit              100040d0     ucrt:api-ms-win-crt-runtime-l1-1-0.dll
 0002:000000d4       __imp___execute_onexit_table 100040d4     ucrt:api-ms-win-crt-runtime-l1-1-0.dll
 0002:000000d8       __imp___initterm           100040d8     ucrt:api-ms-win-crt-runtime-l1-1-0.dll
 0002:000000dc       __imp___initterm_e         100040dc     ucrt:api-ms-win-crt-runtime-l1-1-0.dll
 0002:000000e0       __imp___seh_filter_dll     100040e0     ucrt:api-ms-win-crt-runtime-l1-1-0.dll
 0002:000000e4       __imp___configure_narrow_argv 100040e4     ucrt:api-ms-win-crt-runtime-l1-1-0.dll
 0002:000000e8       __imp___initialize_narrow_environment 100040e8     ucrt:api-ms-win-crt-runtime-l1-1-0.dll
 0002:000000ec       __imp___initialize_onexit_table 100040ec     ucrt:api-ms-win-crt-runtime-l1-1-0.dll
 0002:000000f0       \177api-ms-win-crt-runtime-l1-1-0_NULL_THUNK_DATA 100040f0     ucrt:api-ms-win-crt-runtime-l1-1-0.dll
 0002:000000f4       __imp____acrt_iob_func     100040f4     ucrt:api-ms-win-crt-stdio-l1-1-0.dll
 0002:000000f8       __imp____stdio_common_vfprintf 100040f8     ucrt:api-ms-win-crt-stdio-l1-1-0.dll
 0002:000000fc       __imp____stdio_common_vsprintf 100040fc     ucrt:api-ms-win-crt-stdio-l1-1-0.dll
 0002:00000100       \177api-ms-win-crt-stdio-l1-1-0_NULL_THUNK_DATA 10004100     ucrt:api-ms-win-crt-stdio-l1-1-0.dll
 0002:00000104       __imp__strcpy              10004104     ucrt:api-ms-win-crt-string-l1-1-0.dll
 0002:00000108       __imp__strncmp             10004108     ucrt:api-ms-win-crt-string-l1-1-0.dll
 0002:0000010c       __imp__strlen              1000410c     ucrt:api-ms-win-crt-string-l1-1-0.dll
 0002:00000110       __imp__strcat              10004110     ucrt:api-ms-win-crt-string-l1-1-0.dll
 0002:00000114       \177api-ms-win-crt-string-l1-1-0_NULL_THUNK_DATA 10004114     ucrt:api-ms-win-crt-string-l1-1-0.dll
 0002:00000118       ___guard_check_icall_fptr  10004118     MSVCRT:guard_support.obj
 0002:0000011c       ___castguard_check_failure_os_handled_fptr 1000411c     MSVCRT:guard_support.obj
 0002:00000120       ___xc_a                    10004120     MSVCRT:initializers.obj
 0002:00000124       ___xc_z                    10004124     MSVCRT:initializers.obj
 0002:00000128       ___xi_a                    10004128     MSVCRT:initializers.obj
 0002:0000012c       ___xi_z                    1000412c     MSVCRT:initializers.obj
 0002:00000130       ___xp_a                    10004130     MSVCRT:initializers.obj
 0002:00000134       ___xp_z                    10004134     MSVCRT:initializers.obj
 0002:00000138       ___xt_a                    10004138     MSVCRT:initializers.obj
 0002:0000013c       ___xt_z                    1000413c     MSVCRT:initializers.obj
 0002:00000140       ??_C@_02LMMGGCAJ@?3?5@     10004140     socketTransport.obj
 0002:00000144       ??_C@_0BP@DIBLKMHJ@setsockopt?5SO_REUSEADDR?5failed@ 10004144     socketTransport.obj
 0002:00000164       ??_C@_0BN@KHJBBJDI@setsockopt?5TCPNODELAY?5failed@ 10004164     socketTransport.obj
 0002:00000184       ??_C@_0P@FPMMELAG@JDWP?9Handshake@ 10004184     socketTransport.obj
 0002:00000194       ??_C@_0BJ@GINIINMB@timeout?5during?5handshake@ 10004194     socketTransport.obj
 0002:000001b0       ??_C@_0DC@PHHFHFJN@handshake?5failed?5?9?5connection?5p@ 100041b0     socketTransport.obj
 0002:000001e4       ??_C@_0BN@NDCFIPML@recv?5failed?5during?5handshake@ 100041e4     socketTransport.obj
 0002:00000204       ??_C@_0DB@KBPJCIBD@handshake?5failed?5?9?5received?5?$DO?$CFs@ 10004204     socketTransport.obj
 0002:00000238       ??_C@_0BN@MCHFOAHG@send?5failed?5during?5handshake@ 10004238     socketTransport.obj
 0002:00000258       ??_C@_0O@BNNCBLEN@out?5of?5memory@ 10004258     socketTransport.obj
 0002:00000268       ??_C@_0BM@NGLOKOFN@gethostbyname?3?5unknown?5host@ 10004268     socketTransport.obj
 0002:00000284       ??_C@_01GBGANLPD@0@        10004284     socketTransport.obj
 0002:00000288       ??_C@_0BH@HKLPKFAI@socket?5creation?5failed@ 10004288     socketTransport.obj
 0002:000002a0       ??_C@_0M@NNJMLKEI@bind?5failed@ 100042a0     socketTransport.obj
 0002:000002ac       ??_C@_0O@MHKNJCGE@listen?5failed@ 100042ac     socketTransport.obj
 0002:000002bc       ??_C@_02DPKJAMEF@?$CFd@    100042bc     socketTransport.obj
 0002:000002c0       ??_C@_0M@GKCHHBEN@poll?5failed@ 100042c0     socketTransport.obj
 0002:000002cc       ??_C@_0CB@LPJGLJKP@timed?5out?5waiting?5for?5connectio@ 100042cc     socketTransport.obj
 0002:000002f0       ??_C@_0O@NBABPAKN@accept?5failed@ 100042f0     socketTransport.obj
 0002:00000300       ??_C@_0BP@FADEKCPP@Debugger?5failed?5to?5attach?3?5?$CFs?6@ 10004300     socketTransport.obj
 0002:00000320       ??_C@_0CI@IHMKOBEI@timeout?5waiting?5for?5debugger?5to@ 10004320     socketTransport.obj
 0002:00000348       ??_C@_0BE@KOKKGIKP@connection?5not?5open@ 10004348     socketTransport.obj
 0002:0000035c       ??_C@_0N@NOKLILHD@close?5failed@ 1000435c     socketTransport.obj
 0002:0000036c       ??_C@_0BD@CJKAJNDH@address?5is?5missing@ 1000436c     socketTransport.obj
 0002:00000380       ??_C@_0BI@PPNDHPPD@unable?5to?5create?5socket@ 10004380     socketTransport.obj
 0002:00000398       ??_C@_0BC@DJFNFCAI@connect?5timed?5out@ 10004398     socketTransport.obj
 0002:000003ac       ??_C@_0P@FKKLKLOM@connect?5failed@ 100043ac     socketTransport.obj
 0002:000003bc       ??_C@_0P@KCFPLCED@packet?5is?5NULL@ 100043bc     socketTransport.obj
 0002:000003cc       ??_C@_0P@BHAFPBHF@invalid?5length@ 100043cc     socketTransport.obj
 0002:000003dc       ??_C@_0M@EADLIJBM@send?5failed@ 100043dc     socketTransport.obj
 0002:000003e8       ??_C@_0P@GOGFFADL@packet?5is?5null@ 100043e8     socketTransport.obj
 0002:000003f8       ??_C@_0O@NBMIKEGI@premature?5EOF@ 100043f8     socketTransport.obj
 0002:00000408       ??_C@_0L@IBALKEMH@recv?5error@ 10004408     socketTransport.obj
 0002:00000414       ??_C@_0CO@MNFHICJC@Badly?5formed?5packet?5received?5?9?5@ 10004414     socketTransport.obj
 0002:000005b8       ??_C@_0DE@NDGANADE@Provider?5initialization?5failed?5@ 100045b8     socket_md.obj
 0002:000005ec       ??_C@_0BC@HFNFNKAI@Permission?5denied@ 100045ec     socket_md.obj
 0002:00000600       ??_C@_0BH@LOKACPE@Address?5already?5in?5use@ 10004600     socket_md.obj
 0002:00000618       ??_C@_0CA@NBHADPNL@Cannot?5assign?5requested?5address@ 10004618     socket_md.obj
 0002:00000638       ??_C@_0DA@KDGLCJJO@Address?5family?5not?5supported?5by@ 10004638     socket_md.obj
 0002:00000668       ??_C@_0BO@BMABNIPB@Operation?5already?5in?5progress@ 10004668     socket_md.obj
 0002:00000688       ??_C@_0CB@DJAOADN@Software?5caused?5connection?5abor@ 10004688     socket_md.obj
 0002:000006ac       ??_C@_0BD@NPDMPPFP@Connection?5refused@ 100046ac     socket_md.obj
 0002:000006c0       ??_C@_0BJ@FJAMCHKE@Connection?5reset?5by?5peer@ 100046c0     socket_md.obj
 0002:000006dc       ??_C@_0BN@HFCIEIME@Destination?5address?5required@ 100046dc     socket_md.obj
 0002:000006fc       ??_C@_0M@LOEHLCJD@Bad?5address@ 100046fc     socket_md.obj
 0002:00000708       ??_C@_0N@OHOPOBEF@Host?5is?5down@ 10004708     socket_md.obj
 0002:00000718       ??_C@_0BB@PFBILCPA@No?5route?5to?5host@ 10004718     socket_md.obj
 0002:0000072c       ??_C@_0BK@LBMNDGCG@Operation?5now?5in?5progress@ 1000472c     socket_md.obj
 0002:00000748       ??_C@_0BK@FJBOAFDK@Interrupted?5function?5call@ 10004748     socket_md.obj
 0002:00000764       ??_C@_0BB@HMGGCEBG@Invalid?5argument@ 10004764     socket_md.obj
 0002:00000778       ??_C@_0BM@CCONNCKE@Socket?5is?5already?5connected@ 10004778     socket_md.obj
 0002:00000794       ??_C@_0BE@INBJMKGG@Too?5many?5open?5files@ 10004794     socket_md.obj
 0002:000007a8       ??_C@_0EN@MMGGBIMI@The?5message?5is?5larger?5than?5the?5@ 100047a8     socket_md.obj
 0002:000007f8       ??_C@_0BA@LPIEBGEK@Network?5is?5down@ 100047f8     socket_md.obj
 0002:00000808       ??_C@_0CE@JHDCOCF@Network?5dropped?5connection?5on?5r@ 10004808     socket_md.obj
 0002:0000082c       ??_C@_0BH@CIEOBPFM@Network?5is?5unreachable@ 1000482c     socket_md.obj
 0002:00000844       ??_C@_0DJ@FJOKEEBP@No?5buffer?5space?5available?5?$CImaxi@ 10004844     socket_md.obj
 0002:00000880       ??_C@_0BE@NEGCDJON@Bad?5protocol?5option@ 10004880     socket_md.obj
 0002:00000894       ??_C@_0BI@ILAOGBJJ@Socket?5is?5not?5connected@ 10004894     socket_md.obj
 0002:000008ac       ??_C@_0BO@PFGGHOGH@Socket?5operation?5on?5nonsocket@ 100048ac     socket_md.obj
 0002:000008cc       ??_C@_0BI@EDJAHLMH@Operation?5not?5supported@ 100048cc     socket_md.obj
 0002:000008e4       ??_C@_0BO@EBCCBLCJ@Protocol?5family?5not?5supported@ 100048e4     socket_md.obj
 0002:00000904       ??_C@_0BD@LPHIGPM@Too?5many?5processes@ 10004904     socket_md.obj
 0002:00000918       ??_C@_0BH@JNBKLLAJ@Protocol?5not?5supported@ 10004918     socket_md.obj
 0002:00000930       ??_C@_0BP@PDKJLOAE@Protocol?5wrong?5type?5for?5socket@ 10004930     socket_md.obj
 0002:00000950       ??_C@_0CC@DAIJOIKC@Cannot?5send?5after?5socket?5shutdo@ 10004950     socket_md.obj
 0002:00000974       ??_C@_0BK@LMAIHBL@Socket?5type?5not?5supported@ 10004974     socket_md.obj
 0002:00000990       ??_C@_0BF@IBBHAGLD@Connection?5timed?5out@ 10004990     socket_md.obj
 0002:000009a8       ??_C@_0BF@EHICFGGJ@Class?5type?5not?5found@ 100049a8     socket_md.obj
 0002:000009c0       ??_C@_0CB@EPFKGNAK@Resource?5temporarily?5unavailabl@ 100049c0     socket_md.obj
 0002:000009e4       ??_C@_0P@CAFMJNJH@Host?5not?5found@ 100049e4     socket_md.obj
 0002:000009f4       ??_C@_0BO@GICNLCFB@Insufficient?5memory?5available@ 100049f4     socket_md.obj
 0002:00000a14       ??_C@_0CI@CFJNLLNI@Successful?5WSAStartup?5not?5yet?5p@ 10004a14     socket_md.obj
 0002:00000a3c       ??_C@_0CN@KFPNHBIN@Valid?5name?0?5no?5data?5record?5of?5r@ 10004a3c     socket_md.obj
 0002:00000a6c       ??_C@_0BP@BOOHLDLA@This?5is?5a?5nonrecoverable?5error@ 10004a6c     socket_md.obj
 0002:00000a8c       ??_C@_0CB@PLJNFILF@Network?5subsystem?5is?5unavailabl@ 10004a8c     socket_md.obj
 0002:00000ab0       ??_C@_0CA@DOKOCCFB@Nonauthoritative?5host?5not?5found@ 10004ab0     socket_md.obj
 0002:00000ad0       ??_C@_0CB@GHMLGJBG@Winsock?4dll?5version?5out?5of?5rang@ 10004ad0     socket_md.obj
 0002:00000af4       ??_C@_0BO@ILFFGILJ@Graceful?5shutdown?5in?5progress@ 10004af4     socket_md.obj
 0002:00000b14       ??_C@_0BN@KGMIDOOK@Overlapped?5operation?5aborted@ 10004b14     socket_md.obj
 0002:00000b34       ??_C@_03FCLDNGNL@TCP@      10004b34     socket_md.obj
 0002:00000b38       ??_C@_0BB@IDELEPKG@winsock?5error?5?$CFd@ 10004b38     socket_md.obj
 0002:00000b54       __pDefaultRawDllMain       10004b54     MSVCRT:dll_dllmain.obj
 0002:00000b54       __pRawDllMain              10004b54     MSVCRT:dll_dllmain.obj
 0002:00000b58       __load_config_used         10004b58     MSVCRT:loadcfg.obj
 0002:00000c80       ___safe_se_handler_table   10004c80     <linker-defined>
 0002:00000c84       ___volatile_metadata       10004c84     <linker-defined>
 0002:00000fe0       ___rtc_iaa                 10004fe0     MSVCRT:initsect.obj
 0002:00000fe4       ___rtc_izz                 10004fe4     MSVCRT:initsect.obj
 0002:00000fe8       ___rtc_taa                 10004fe8     MSVCRT:initsect.obj
 0002:00000fec       ___rtc_tzz                 10004fec     MSVCRT:initsect.obj
 0002:000010d8       __IMPORT_DESCRIPTOR_WS2_32 100050d8     ws2_32:WS2_32.dll
 0002:000010ec       __IMPORT_DESCRIPTOR_KERNEL32 100050ec     kernel32:KERNEL32.dll
 0002:00001100       __IMPORT_DESCRIPTOR_VCRUNTIME140 10005100     vcruntime:VCRUNTIME140.dll
 0002:00001114       __IMPORT_DESCRIPTOR_api-ms-win-crt-stdio-l1-1-0 10005114     ucrt:api-ms-win-crt-stdio-l1-1-0.dll
 0002:00001128       __IMPORT_DESCRIPTOR_api-ms-win-crt-string-l1-1-0 10005128     ucrt:api-ms-win-crt-string-l1-1-0.dll
 0002:0000113c       __IMPORT_DESCRIPTOR_api-ms-win-crt-convert-l1-1-0 1000513c     ucrt:api-ms-win-crt-convert-l1-1-0.dll
 0002:00001150       __IMPORT_DESCRIPTOR_api-ms-win-crt-runtime-l1-1-0 10005150     ucrt:api-ms-win-crt-runtime-l1-1-0.dll
 0002:00001164       __NULL_IMPORT_DESCRIPTOR   10005164     ws2_32:WS2_32.dll
 0003:00000008       ___security_cookie_complement 10006008     MSVCRT:gs_cookie.obj
 0003:0000000c       ___security_cookie         1000600c     MSVCRT:gs_cookie.obj
 0003:00000010       ___scrt_native_dllmain_reason 10006010     MSVCRT:utility.obj
 0003:00000020       ___isa_enabled             10006020     MSVCRT:cpu_disp.obj
 0003:00000024       ___scrt_ucrt_dll_is_in_use 10006024     MSVCRT:ucrt_stubs.obj
 0003:00000390       ?__type_info_root_node@@3U__type_info_node@@A 10006390     MSVCRT:tncleanup.obj
 0003:00000398       ?_OptionsStorage@?1??__local_stdio_scanf_options@@9@4_KA 10006398     MSVCRT:default_local_stdio_options.obj
 0003:000003a0       ___scrt_current_native_startup_state 100063a0     MSVCRT:utility.obj
 0003:000003a4       ___scrt_native_startup_lock 100063a4     MSVCRT:utility.obj
 0003:000003c4       ___scrt_debugger_hook_flag 100063c4     MSVCRT:utility_desktop.obj
 0003:000003c8       ___isa_available           100063c8     MSVCRT:cpu_disp.obj
 0003:000003cc       ___favor                   100063cc     MSVCRT:cpu_disp.obj
 0003:000003d0       ?_OptionsStorage@?1??__local_stdio_printf_options@@9@9 100063d0     <common>
 0003:000003d8       ___dyn_tls_init_callback   100063d8     <common>

 entry point at        0001:0000195a

 Static symbols

 0000:ffff7000       .debug$S                   10000000     dt_socket.exp
 0000:ffff7000       .debug$S                   10000000     vcruntime:VCRUNTIME140.dll
 0000:ffff7000       .debug$S                   10000000     vcruntime:VCRUNTIME140.dll
 0000:ffff7000       .debug$S                   10000000     vcruntime:VCRUNTIME140.dll
 0000:ffff7000       .debug$S                   10000000     vcruntime:VCRUNTIME140.dll
 0000:ffff7000       .debug$S                   10000000     vcruntime:VCRUNTIME140.dll
 0000:ffff7000       .debug$S                   10000000     vcruntime:VCRUNTIME140.dll
 0000:ffff7000       .debug$S                   10000000     vcruntime:VCRUNTIME140.dll
 0000:ffff7000       .debug$S                   10000000     ucrt:api-ms-win-crt-convert-l1-1-0.dll
 0000:ffff7000       .debug$S                   10000000     ucrt:api-ms-win-crt-runtime-l1-1-0.dll
 0000:ffff7000       .debug$S                   10000000     ucrt:api-ms-win-crt-runtime-l1-1-0.dll
 0000:ffff7000       .debug$S                   10000000     ucrt:api-ms-win-crt-runtime-l1-1-0.dll
 0000:ffff7000       .debug$S                   10000000     ucrt:api-ms-win-crt-runtime-l1-1-0.dll
 0000:ffff7000       .debug$S                   10000000     ucrt:api-ms-win-crt-runtime-l1-1-0.dll
 0000:ffff7000       .debug$S                   10000000     ucrt:api-ms-win-crt-runtime-l1-1-0.dll
 0000:ffff7000       .debug$S                   10000000     ucrt:api-ms-win-crt-runtime-l1-1-0.dll
 0000:ffff7000       .debug$S                   10000000     ucrt:api-ms-win-crt-runtime-l1-1-0.dll
 0000:ffff7000       .debug$S                   10000000     ucrt:api-ms-win-crt-runtime-l1-1-0.dll
 0000:ffff7000       .debug$S                   10000000     ucrt:api-ms-win-crt-runtime-l1-1-0.dll
 0000:ffff7000       .debug$S                   10000000     ucrt:api-ms-win-crt-runtime-l1-1-0.dll
 0000:ffff7000       .debug$S                   10000000     ucrt:api-ms-win-crt-runtime-l1-1-0.dll
 0000:ffff7000       .debug$S                   10000000     ucrt:api-ms-win-crt-stdio-l1-1-0.dll
 0000:ffff7000       .debug$S                   10000000     ucrt:api-ms-win-crt-stdio-l1-1-0.dll
 0000:ffff7000       .debug$S                   10000000     ucrt:api-ms-win-crt-stdio-l1-1-0.dll
 0000:ffff7000       .debug$S                   10000000     ucrt:api-ms-win-crt-string-l1-1-0.dll
 0000:ffff7000       .debug$S                   10000000     ucrt:api-ms-win-crt-string-l1-1-0.dll
 0000:ffff7000       .debug$S                   10000000     ucrt:api-ms-win-crt-string-l1-1-0.dll
 0000:ffff7000       .debug$S                   10000000     ucrt:api-ms-win-crt-string-l1-1-0.dll
 0000:ffff7000       .debug$S                   10000000     kernel32:KERNEL32.dll
 0000:ffff7000       .debug$S                   10000000     kernel32:KERNEL32.dll
 0000:ffff7000       .debug$S                   10000000     kernel32:KERNEL32.dll
 0000:ffff7000       .debug$S                   10000000     kernel32:KERNEL32.dll
 0000:ffff7000       .debug$S                   10000000     kernel32:KERNEL32.dll
 0000:ffff7000       .debug$S                   10000000     kernel32:KERNEL32.dll
 0000:ffff7000       .debug$S                   10000000     kernel32:KERNEL32.dll
 0000:ffff7000       .debug$S                   10000000     kernel32:KERNEL32.dll
 0000:ffff7000       .debug$S                   10000000     kernel32:KERNEL32.dll
 0000:ffff7000       .debug$S                   10000000     kernel32:KERNEL32.dll
 0000:ffff7000       .debug$S                   10000000     kernel32:KERNEL32.dll
 0000:ffff7000       .debug$S                   10000000     kernel32:KERNEL32.dll
 0000:ffff7000       .debug$S                   10000000     kernel32:KERNEL32.dll
 0000:ffff7000       .debug$S                   10000000     kernel32:KERNEL32.dll
 0000:ffff7000       .debug$S                   10000000     kernel32:KERNEL32.dll
 0000:ffff7000       .debug$S                   10000000     kernel32:KERNEL32.dll
 0000:ffff7000       .debug$S                   10000000     kernel32:KERNEL32.dll
 0000:ffff7000       .debug$S                   10000000     kernel32:KERNEL32.dll
 0000:ffff7000       .debug$S                   10000000     kernel32:KERNEL32.dll
 0000:ffff7000       .debug$S                   10000000     kernel32:KERNEL32.dll
 0000:ffff7000       .debug$S                   10000000     ws2_32:WS2_32.dll
 0000:ffff7000       .debug$S                   10000000     ws2_32:WS2_32.dll
 0000:ffff7000       .debug$S                   10000000     ws2_32:WS2_32.dll
 0000:ffff7000       .debug$S                   10000000     ws2_32:WS2_32.dll
 0000:ffff7000       .debug$S                   10000000     ws2_32:WS2_32.dll
 0000:ffff7000       .debug$S                   10000000     ws2_32:WS2_32.dll
 0000:ffff7000       .debug$S                   10000000     ws2_32:WS2_32.dll
 0000:ffff7000       .debug$S                   10000000     ws2_32:WS2_32.dll
 0000:ffff7000       .debug$S                   10000000     ws2_32:WS2_32.dll
 0000:ffff7000       .debug$S                   10000000     ws2_32:WS2_32.dll
 0000:ffff7000       .debug$S                   10000000     ws2_32:WS2_32.dll
 0000:ffff7000       .debug$S                   10000000     ws2_32:WS2_32.dll
 0000:ffff7000       .debug$S                   10000000     ws2_32:WS2_32.dll
 0000:ffff7000       .debug$S                   10000000     ws2_32:WS2_32.dll
 0000:ffff7000       .debug$S                   10000000     ws2_32:WS2_32.dll
 0000:ffff7000       .debug$S                   10000000     ws2_32:WS2_32.dll
 0000:ffff7000       .debug$S                   10000000     ws2_32:WS2_32.dll
 0000:ffff7000       .debug$S                   10000000     ws2_32:WS2_32.dll
 0000:ffff7000       .debug$S                   10000000     ws2_32:WS2_32.dll
 0000:ffff7000       .debug$S                   10000000     ws2_32:WS2_32.dll
 0000:ffff7000       .debug$S                   10000000     ws2_32:WS2_32.dll
 0000:ffff7000       .debug$S                   10000000     ws2_32:WS2_32.dll
 0000:ffff7000       .debug$S                   10000000     ws2_32:WS2_32.dll
 0000:ffff7000       .debug$S                   10000000     ws2_32:WS2_32.dll
 0000:ffff7000       .debug$S                   10000000     ws2_32:WS2_32.dll
 0000:ffff7000       .debug$S                   10000000     ws2_32:WS2_32.dll
 0000:ffff7000       .debug$S                   10000000     ws2_32:WS2_32.dll
 0001:00000075       _handshake                 10001075 f   socketTransport.obj
 0001:0000029c       _parseAddress              1000129c f   socketTransport.obj
 0001:000003a8       _recv_fully                100013a8 f   socketTransport.obj
 0001:000003e1       _send_fully                100013e1 f   socketTransport.obj
 0001:0000041a       _setLastError              1000141a f   socketTransport.obj
 0001:000004fd       _setOptions                100014fd f   socketTransport.obj
 0001:00000555       _socketTransport_accept@20 10001555 f   socketTransport.obj
 0001:00000750       _socketTransport_attach@24 10001750 f   socketTransport.obj
 0001:000008c9       _socketTransport_close@4   100018c9 f   socketTransport.obj
 0001:00000901       _socketTransport_getCapabilities@8 10001901 f   socketTransport.obj
 0001:00000926       _socketTransport_getLastError@8 10001926 f   socketTransport.obj
 0001:0000096f       _socketTransport_isOpen@4  1000196f f   socketTransport.obj
 0001:0000097c       _socketTransport_readPacket@8 1000197c f   socketTransport.obj
 0001:00000afa       _socketTransport_startListening@12 10001afa f   socketTransport.obj
 0001:00000c50       _socketTransport_stopListening@4 10001c50 f   socketTransport.obj
 0001:00000c94       _socketTransport_writePacket@8 10001c94 f   socketTransport.obj
 0001:00001570       $$000000                   10002570     MSVCRT:lldiv.obj
 0001:00001591       L1                         10002591     MSVCRT:lldiv.obj
 0001:000015ad       L2                         100025ad     MSVCRT:lldiv.obj
 0001:000015c9       L3                         100025c9     MSVCRT:lldiv.obj
 0001:000015d7       L5                         100025d7     MSVCRT:lldiv.obj
 0001:00001605       L6                         10002605     MSVCRT:lldiv.obj
 0001:00001606       L7                         10002606     MSVCRT:lldiv.obj
 0001:0000160a       L4                         1000260a     MSVCRT:lldiv.obj
 0001:00001614       L8                         10002614     MSVCRT:lldiv.obj
 0001:0000161a       ?dllmain_crt_dispatch@@YGHQAUHINSTANCE__@@KQAX@Z 1000261a f   MSVCRT:dll_dllmain.obj
 0001:0000166d       ?dllmain_crt_process_attach@@YAHQAUHINSTANCE__@@QAX@Z 1000266d f   MSVCRT:dll_dllmain.obj
 0001:00001774       ?dllmain_crt_process_detach@@YAH_N@Z 10002774 f   MSVCRT:dll_dllmain.obj
 0001:00001824       ?dllmain_dispatch@@YAHQAUHINSTANCE__@@KQAX@Z 10002824 f   MSVCRT:dll_dllmain.obj
 0001:0000192f       ?dllmain_raw@@YGHQAUHINSTANCE__@@KQAX@Z 1000292f f   MSVCRT:dll_dllmain.obj
 0001:0000197d       ___get_entropy             1000297d f   MSVCRT:gs_support.obj
 0001:00001a50       ?find_pe_section@@YAPAU_IMAGE_SECTION_HEADER@@QAEI@Z 10002a50 f   MSVCRT:utility.obj
 0001:00001eb0       $$000000                   10002eb0     MSVCRT:sehprolg4.obj
 0002:00000448       _winsock_errors            10004448     socket_md.obj
 0002:00000b4c       _GS_ExceptionPointers      10004b4c     MSVCRT:gs_report.obj
 0002:00000ff0       __sehtable$?dllmain_crt_process_attach@@YAHQAUHINSTANCE__@@QAX@Z 10004ff0     MSVCRT:dll_dllmain.obj
 0002:00001010       __sehtable$?dllmain_crt_process_detach@@YAH_N@Z 10005010     MSVCRT:dll_dllmain.obj
 0002:00001038       __sehtable$?dllmain_dispatch@@YAHQAUHINSTANCE__@@KQAX@Z 10005038     MSVCRT:dll_dllmain.obj
 0002:00001058       __sehtable$___scrt_is_nonwritable_in_current_image 10005058     MSVCRT:utility.obj
 0002:00001080       .edata                     10005080     dt_socket.exp
 0002:000010a8       rgpv                       100050a8     dt_socket.exp
 0002:000010ac       rgszName                   100050ac     dt_socket.exp
 0002:000010b0       rgwOrd                     100050b0     dt_socket.exp
 0002:000010b2       szName                     100050b2     dt_socket.exp
 0002:000010c0       $N00001                    100050c0     dt_socket.exp
 0002:000012a4       .idata$6                   100052a4     ws2_32:WS2_32.dll
 0002:00001420       .idata$6                   10005420     kernel32:KERNEL32.dll
 0002:00001486       .idata$6                   10005486     vcruntime:VCRUNTIME140.dll
 0002:000015b4       .idata$6                   100055b4     ucrt:api-ms-win-crt-stdio-l1-1-0.dll
 0002:000015d4       .idata$6                   100055d4     ucrt:api-ms-win-crt-string-l1-1-0.dll
 0002:000015f6       .idata$6                   100055f6     ucrt:api-ms-win-crt-convert-l1-1-0.dll
 0002:00001618       .idata$6                   10005618     ucrt:api-ms-win-crt-runtime-l1-1-0.dll
 0003:00000000       _socketFD                  10006000     socketTransport.obj
 0003:00000004       _single_env                10006004     socketTransport.obj
 0003:00000028       _interface                 10006028     socketTransport.obj
 0003:00000054       _serverSocketFD            10006054     socketTransport.obj
 0003:00000058       _callback                  10006058     socketTransport.obj
 0003:0000005c       _jvm                       1000605c     socketTransport.obj
 0003:00000060       _tlsIndex                  10006060     socketTransport.obj
 0003:00000064       _initialized               10006064     socketTransport.obj
 0003:00000068       ?fileTime_1_1_70@?1??dbgsysCurrentTimeMillis@@9@9 10006068     socket_md.obj
 0003:00000070       _GS_ExceptionRecord        10006070     MSVCRT:gs_report.obj
 0003:000000c0       _GS_ContextRecord          100060c0     MSVCRT:gs_report.obj
 0003:0000038c       ?__proc_attached@@3HA      1000638c     MSVCRT:dll_dllmain.obj
 0003:000003a8       ?is_initialized_as_dll@@3_NA 100063a8     MSVCRT:utility.obj
 0003:000003a9       ?module_local_atexit_table_initialized@@3_NA 100063a9     MSVCRT:utility.obj
 0003:000003ac       ?module_local_atexit_table@@3U_onexit_table_t@@A 100063ac     MSVCRT:utility.obj
 0003:000003b8       ?module_local_at_quick_exit_table@@3U_onexit_table_t@@A 100063b8     MSVCRT:utility.obj
 0004:00000060       $R000000                   10007060     dt_socket.dll.res
